:03000000020AD819
:0C0AD800787FE4F6D8FD758153020B1FF7
:100F7A00545820202020202020202020205A5A4E59
:100F8A00003138313130353033352020202E20439E
:020F9A00440011
:100EF900C2B17F017E00120F0A8B80D2B27F017EC0
:010F090000E7
:100F0A00D3EF9400EE940040147D6E7C00ED1D70CA
:0D0F1A00011CED4C70F7EF1F70E61E80E328
:010F270022A7
:091087007F057E00120F0A7F387C
:0C109000AB07C2B2C2B0120EF9C2B2220D
:0C10B000AB07C2B2D2B0120EF9C2B222DD
:100E33007F381210901210871210877F08121090BB
:100E43007F011210907F061210907F0C1210907F7A
:100E530080121090E4FAEA900F7A93FF1210B00A0E
:100E6300BA10F37FC0121090E4FAEA900F8B93FF4D
:070E73001210B00ABA10F3DF
:010E7A002255
:100FDD00C2A77F677E00EF1F70011EEF4E70F7D224
:0E0FED00A77E007F04EF1F70011EEF4E70F70D
:010FFB0022D3
:100F5600C2A70FBF0000D2A70FBF00000FBF00003F
:100F6600A2A792007E007F08EF1F70011EEF4E7051
:030F7600F7A200DF
:010F79002255
:10101A00E4FD7C01120F56E433FFC43333335480AA
:0C102A00FEEDC3134EFD0CBC09EAAF053F
:011036002297
:10105300C2A70FBF00000FBF0000D2A77E007F080A
:09106300EF1F70011EEF4E70F743
:01106C002261
:10106D00C2A77F087E00EF1F70011EEF4E70F7D2F2
:09107D00A70FBF00000FBF000027
:011086002247
:02103700AD0703
:101039007B01ED139200EDC313FD3000051210532F
:09104900800312106D0BBB09E9D4
:01105200227B
:10109C00120FDD7F017E00120F0A7FCC1210377FFA
:0410AC0044021037B3
:100D4000120FDD7F017E00120F0A7FCC1210377F59
:100D5000BE12103712101AAB0712101AEFFEEBFF7B
:100D6000FDAC06E4120832E4FBFA7980783D120704
:100D7000278F0B8E0A8D098C08E4FFFE7D207C41B5
:100D8000AB0BAA0AA909A808120727E4FBFAF9780D
:070D90003F12063612086B4A
:010D97002239
:100D98002020482F4C3D302F313A2020202020435E
:100DA800004F2F443A2020202020202020202020DF
:100DB8004300303132333435363738393A4D61787B
:100DC8002020202020202020202E204344004D6970
:0F0DD8006E2020202020202020202E20434400A9
:100FBD00023D00010242000102460001024A000109
:0F0FCD00024E00010250000102520001012500F6
:0B10BC00EF1FAC0670011E4C70F62206
:060CE5008D0BAB07AA060F
:100CEB007C007D641208FE8F0C7C007D64AF03AE2C
:100CFB00021208FE7E007F0ACFCDCFCECCCE1208DB
:100D0B00FE8F0DAE02AF037C007D0A1208FE8D0E26
:100D1B00AF0B121090E50C2430FF1210B0E50D2430
:100D2B0030FF1210B0E50B2403FF121090E50E24D8
:050D3B0030FF0210B0C2
:100BC7007F381210907F057E00120F0A7F381210AF
:100BD700907F057E00120F0A7F381210907F08124F
:100BE70010907F011210907F061210907F0C121048
:100BF700907F801210907FC0121090E4F50AE50AEA
:100C0700900DD693FF1210B0050AE50AC394104061
:100C1700ED7DCAAF22AE21120CE57F007EF20210F5
:010C2700BC10
:100C28007F381210907F057E00120F0A7F3812104D
:100C3800907F057E00120F0A7F381210907F0812ED
:100C480010907F011210907F061210907F0C1210E6
:100C5800907F801210907FC0121090E4F50AE50A88
:100C6800900DC593FF1210B0050AE50AC394104011
:100C7800ED7DCAAF24AE23120CE57F007EF2021090
:010C8800BCAF
:070F9C00900DBA93FBE4FD88
:100FA3008F0E8B0FED7006E50E24808004E50E2472
:0A0FB300C0FF121090AF0F0210B043
:100B64008D098B0AEF7F04120F9CE5097F05120F94
:100B74009C900DC4E493FBE4FD7F06120FA3E50AE9
:100B8400900DBA93FBE4FD7F07120FA3E50B900DC4
:100B9400BA93FBE4FD7F08120FA3900DC4E493FB0A
:100BA400E4FD7F09120FA3E50C900DBA93FBE4FD5D
:100BB4007F0A120FA3E50D900DBA93FBE4FD7F0BA2
:030BC400020FA37A
:060DE7007D8BAF28AE2752
:060DED008D0AAB07AA0607
:100DF3007C007D641208FE8F0BAE02AF037C007D86
:100E0300641208FE7E007F0ACFCDCFCECCCE12086F
:100E1300FE8F0CAF0A121090E50C2430FF1210B0B5
:100E2300E50B2430FF1210B0E50A2403FF021090F3
:060FFC007DCAAF2AAE29F8
:02100200AB053C
:101004007C007D0A1208FE8D0AAF03121090E50AD7
:061014002430FF0210B0C1
:10001E007F80121090E4F508E508900D9893FF127A
:10002E0010B00508E508C3941040ED7FC012109083
:10003E00E4F509E509900DA993FF1210B00509E545
:10004E0009C3941040EDE525700302062C120DE74E
:10005E00120FFCE52560EF24FE600F14600A146099
:10006E001914601B2404701C80047F8B80027FCACD
:10007E001210907F0F121090800D120C2880081213
:10008E000BC78003E4F525309103020171E5256469
:10009E000160030201717F32FE120F0AE4F544F58E
:1000AE00457D80AF45AE441210027FD512109030C0
:1000BE0091030201717F0A7E00120F0A053EE53E92
:1000CE007002053D3091FDAE3DAF3E7C007D0B12C2
:1000DE000953EC6003020171ED14B40A00400302EF
:1000EE0001719000FE75F003A4C58325F0C58373DE
:1000FE0002011C02012302012B02013302013B0209
:10010E00014302014B02015302015B020163E4F55C
:10011E0029F52A8046752900752A01803E75290029
:10012E00752A028036752900752A03802E752900DE
:10013E00752A048026752900752A05801E752900EA
:10014E00752A068016752900752A07800E752900F6
:10015E00752A088006752900752A09120FFC7FD5AD
:10016E00121090309003020254E5256401600302E0
:10017E0002547F32FE120F0A7544007545017D80D0
:10018E00AF45AE441210027FD5121090309003028C
:10019E0002547F0A7E00120F0A054BE54B700205D2
:1001AE004A3090FDAE4AAF4B7C007D0B120953ECEA
:1001BE006003020254ED14B40A004003020254908C
:1001CE0001DB75F003A4C58325F0C583730201F925
:1001DE0002020002020802021002021802022002AB
:1001EE000228020230020238020240E4F534F535EC
:1001FE008046753400753501803E753400753502C4
:10020E008036753400753503802E753400753504CF
:10021E008026753400753505801E753400753506DB
:10022E008016753400753507800E753400753508E7
:10023E0080067534007535097DCAAF35AE3412109F
:10024E00027FD5121090309103020329E525640236
:10025E0060030203297F0AFE120F0AE4F53FF54000
:10026E007D80AF40AE3F120DED7F8B12109030911E
:10027E00030203290543E543700205423091FDAEAA
:10028E0042AF437C007D0B120953EC60030203293D
:10029E00ED14B40A0040030203299002B675F00370
:1002AE00A4C58325F0C583730202D40202DB0202C9
:1002BE00E30202EB0202F30202FB02030302030B50
:1002CE0002031302031BE4F527F528804675270069
:1002DE0075280A803E75270075281480367527000C
:1002EE0075281E802E7527007528288026752700F4
:1002FE00752832801E75270075283C8016752700DC
:10030E00752846800E7527007528508006752700C3
:10031E0075285A120DE77F8B12109030900302044D
:10032E0005E525640260030204057F0AFE120F0A2A
:10033E00753F0075400A7D80AF40AE3F120DED7FD8
:10034E008B1210903090030204050547E5477002AA
:10035E0005463090FDAE46AF477C007D0B1209532B
:10036E00EC6003020405ED14B40A00400302040518
:10037E0090038C75F003A4C58325F0C58373020327
:10038E00AA0203B10203B90203C10203C90203D1D7
:10039E000203D90203E10203E90203F1E4F532F5A7
:1003AE0033804675320075330A803E7532007533E0
:1003BE0014803675320075331E802E7532007533FB
:1003CE00288026753200753332801E7532007533E3
:1003DE003C8016753200753346800E7532007533CB
:1003EE0050800675320075335A7D8BAF33AE3212A4
:1003FE000DED7F8B1210903091030204E7E525641A
:10040E000360030204E77F32FE120F0AE4F548F59B
:10041E00497D80AF49AE48120DED7FD51210903058
:10042E0091030204E77F0A7E00120F0A054FE54F83
:10043E007002054E3091FDAE4EAF4F7C007D0B121B
:10044E000953EC60030204E7ED14B40A0040030202
:10045E0004E790046E75F003A4C58325F0C583737D
:10046E0002048C02049302049B0204A30204AB0256
:10047E0004B30204BB0204C30204CB0204D3E4F5AA
:10048E0030F5318046753000753101803E75300093
:10049E007531028036753000753103802E7530004F
:1004AE007531048026753000753105801E7530005B
:1004BE007531068016753000753107800E75300067
:1004CE0075310880067530007531097DCAAF31AEC1
:1004DE00301210027FD51210903090030205CAE53B
:1004EE0025640360030205CA7F32FE120F0A7548A7
:1004FE000075490A7D80AF49AE48120DED7FD512C9
:10050E0010903090030205CA7F0A7E00120F0A0572
:10051E0051E551700205503090FDAE50AF517C0048
:10052E007D0B120953EC60030205CAED14B40A00E8
:10053E0040030205CA90055175F003A4C58325F04A
:10054E00C5837302056F02057602057E02058602DB
:10055E00058E02059602059E0205A60205AE02054F
:10056E00B6E4F54CF54D8046754C00754D01803E58
:10057E00754C00754D028036754C00754D03802EFE
:10058E00754C00754D048026754C00754D05801E0A
:10059E00754C00754D068016754C00754D07800E16
:1005AE00754C00754D088006754C00754D097DCA59
:1005BE00AF4DAE4C1210027FD5121090E525B4044B
:1005CE0029AE29AF2A7C007D0A1208ECAA06AB07D9
:1005DE00AE27AF281208ECEF2BFFEE3AFEE5312FD7
:1005EE00F524E5303EF523120C28E525640560035D
:1005FE00020061AE34AF35FC7D0A1208ECAA06ABE0
:10060E0007AE32AF331208ECEF2BFFEE3AFEE54D9C
:10061E002FF522E54C3EF521120BC7020061020EAA
:01062E003398
:100E7B00120E33D2A1E4F525F527752850F529F587
:100E8B002AF53275330AF534F535F530F531F54C75
:100E9B00F54DD2AFD2AAD2AB758901D28A758DEE40
:100EAB00F58BC28EF526F52CF52DF52B758C3C7537
:070EBB008AB0D28CD2A922FB
:100997007590E7120E7BE525600512001E80F7E5CE
:1009A7002570F37F64FE120F0A12109C120D408E01
:1009B7002E8F2F20951A7F057E00120F0A20950D86
:1009C700E52C64176004052C8003E4F52C3095FDB5
:1009D70020961A7F057E00120F0A20960DE52D64DA
:1009E7003B6004052D8003E4F52D3096FD20971A12
:1009F7007F057E00120F0A20970DE52B643B6004EC
:100A0700052B8003E4F52B3097FDE52C75F00A8460
:100A1700F53AE52C75F00A8485F03BE52D75F00A6B
:100A270084F53CE52D75F00A8485F041E52B75F0DA
:100A37000A84F538E52B75F00A8485F039AE29AFBD
:100A47002A7C007D0A1208ECAA06AB07AE27AF285E
:100A57001208ECEF2BFFEE3AFEE5312FF524E530D7
:100A67003EF523AE34AF351208ECAA06AB07AE321B
:100A7700AF331208ECEF2BFFEE3AFEE54D2FF522D0
:100A8700E54C3EF521C3E52F9524E52E952340043B
:100A9700D28E8011D3E52F9522E52E95215004D2D1
:100AA7008E8002C28E7F0A7E00120F0A7DCAAF2F88
:100AB700AE2E120CE585410B85380C85390DAB3C04
:100AC700AD3BAF3A120B647F647E00120F0A020936
:010AD7009D81
:03001300020C8953
:100C8900C0E0C0F0C083C082C0D075D000C000C031
:100C990001C002C003C004C005C006C0077F327E80
:100CA90000120F0AE5B060077F327E00120F0A05B5
:100CB90025E52575F0078485F0257F327E00120F22
:100CC9000AD007D006D005D004D003D002D001D075
:0C0CD90000D0D0D082D083D0F0D0E03228
:03001B00020F28A9
:100F2800C0E0C0D075D000C004C006C007758DEE03
:100F3800758B00B2A17F017E001210BCD28E209268
:0E0F480002C28ED007D006D004D0D0D0E03246
:03000B00020EC220
:100EC200C0E0C0D0758C3C758AB00526E526B41406
:100ED20021752600052BE52BB43C17752B00052D3B
:100EE200E52DB43C0D752D00052CE52CB4180375C9
:070EF2002C00D0D0D0E0324B
:10062F000208D7E86480F8E933E83360110460F01A
:10063F00ED33EC337009E8FCE9FDEAFEEBFF220431
:10064F0060DED3EB9FEA9EE99DE8C2E78CF0C2F72C
:10065F0095F0400CE8CCF8E9CDF9EACEFAEBCFFBF8
:10066F001208A285D0F05804700320D5B3E80470A7
:10067F00075002B2D50208E192D5EC0460F7E4CC42
:10068F00C0E0C398F8603B94186008400DD0E0FBC1
:10069F000208B9E4FBFAC9FC8028E830E406E4C993
:1006AF00FBE4CAFCE830E305E4C9CACBFCE8540715
:1006BF006010F8C3E913F9EA13FAEB13FBEC13FC20
:1006CF00D8F130F52FC3E49CFCEF9BFFEE9AFEEDC3
:1006DF0099FDD0E0FBEF4E4D4C701222DB03020868
:1006EF00DEEC2CFCEF33FFEE33FEED33FDED30E7A8
:1006FF00EB0208B9EF2BFFEE3AFEED39FDD0E0FB30
:10070F0050130BBB00030208E1ED13FDEE13FEEFD8
:08071F0013FFEC13FC0208B902
:10072700EC4D6011E8497017ED33EC3304600DE4CC
:10073700FCFFFEFD22E933E8330470F80208D71204
:1007470008A258046009E4CC248150062850090205
:1007570008E12840030208DEC0E0EB4A7044B98094
:1007670006D0E0FB0208CDEF4E701CBD8008EBFF02
:10077700EAFEE9FD80EBE98DF0A4FEE5F002081042
:10078700E9CDF9EAFEEBFFEF89F0A4FCE5F0CE89AD
:10079700F0A42EFFE435F0CD89F0A42DFEE435F06A
:1007A7008067EF4E7005BD80D780C3EF8BF0A4AC98
:1007B700F0EE8BF0A42CFCE435F0F8EF8AF0A42CD3
:1007C700E5F038FCE433CB8DF0A42CFCE5F03BF8E6
:1007D700EE8AF0A42CFCE5F038F8E433CF89F0A4D6
:1007E7002CFCE5F038CF3400CE89F0A42FFFE5F0DC
:1007F7003EFEE433C98DF0A42EFEE5F039CD8AF034
:10080700A42FFFE5F03EFEE43DFD33D0E0FB5007AB
:100817000BBB000F0208E1EC2CFCEF33FFEE33FEBD
:06082700ED33FD0208B9EB
:10082D0075F020800E75F010800575F0087D007E46
:10083D00007F003392D530D503120989EC33401077
:10084D00EF33FFEE33FEED33FDEC33FCD5F0ED224F
:0E085D00E5F0247EA2D513CC92E7CDCEFF228B
:10086B00EDD2E7CD33EC3392D524814006E4FFFE85
:10087B00FDFC22FCE4CFCECDCC24E0501174FF80E4
:10088B00EDC3CC13CCCD13CDCE13CECF13CF047081
:07089B00F030D5DE020989EF
:1008A200E9D2E7C933E833F892D5EDD2E7CD33EC9C
:0708B20033FC5002B2D52215
:1008B900EC30E7100FBF000C0EBE00080DBD0004A0
:1008C9000BEB6014A2D5EB13FCED92E7FD2274FF4C
:1008D900FCFDFEFF22E480F8A2D574FF13FC7D80A5
:0308E900E480EFB9
:100AE400020997E493A3F8E493A34003F68001F288
:100AF40008DFF48029E493A3F85407240CC8C33313
:100B0400C4540F4420C8834004F456800146F6DFE1
:100B1400E4800B0102040810204080900FBDE47EA5
:100B2400019360BCA3FF543F30E509541FFEE493D6
:100B3400A360010ECF54C025E060A840B8E493A39D
:100B4400FAE493A3F8E493A3C8C582C8CAC583CAC8
:100B5400F0A3C8C582C8CAC583CADFE9DEE780BE80
:010FDC000014
:1008EC00EF8DF0A4A8F0CF8CF0A428CE8DF0A42E20
:0208FC00FE22DA
:1008FE00BC000BBE0029EF8DF084FFADF022E4CCDE
:10090E00F875F008EF2FFFEE33FEEC33FCEE9DECA6
:10091E00984005FCEE9DFE0FD5F0E9E4CEFD22EDEC
:10092E00F8F5F0EE8420D21CFEADF075F008EF2F36
:10093E00FFED33FD4007985006D5F0F222C398FD27
:05094E000FD5F0EA22C4
:10095300C2D5EC30E709B2D5E4C39DFDE49CFCEEBF
:1009630030E715B2D5E4C39FFFE49EFE1208FEC331
:10097300E49DFDE49CFC80031208FE30D507C3E42C
:060983009FFFE49EFE222E
:0E098900C3E49FFFE49EFEE49DFDE49CFC227F
:00000001FF
